:020000040000FA
:040000006E303A28FC
:08000800A000030EA100831209
:1000100081018B100B11210E8300A00E200E090010
:0C007400203084008001840A6030040207
:10008000031C3C281230B00069218316FF23900026
:10009000831283160C308505870183128501870141
:1000A000073099000030831691008312C830831600
:1000B0008100831231309000003083168C0083124F
:1000C00010308B00831600309B001C141A0883121A
:1000D000BC00831610309B001C141A088312BD004C
:1000E000822181018E018F010B118B100B108C016D
:1000F0008B17892031198B204D21B30B87280310D2
:1001000085190314B90DF03039020319A621AE2167
:10011000792864000800080031110130B7008B1302
:100120002030370783169B001C141A088312A40082
:100130001030370783169B001C141A088312A30083
:100140000030370783169B001C141A088312A20084
:100150008B17321CB12822090339A200A309A40974
:10016000A50901303702031DBA283D18BA283D14ED
:100170003E146A2102303702031DC328BD18C3286C
:10018000BD143E146D2103303702031DCC283D19E8
:10019000CC283D153E14702104303702031DD528AC
:1001A000BD19D528BD153E14732105303702031D36
:1001B000DE283D1ADE283D163E1476210630370231
:1001C000031DE728BD1AE728BD163E147921073024
:1001D0003702031DF0283D1BF0283D173E147C21FB
:1001E00008303702031DF928BD1BF928BD173E143E
:1001F0007F21B70A09303702031808008F28013021
:10020000B600B300B400B500B70085018701B11393
:100210008920B30B2529031085190314B90DF0307B
:10022000390203194329B41F8501B41F8701B40B98
:1002300025293708B6080319B60003192329FF300A
:1002400085008700B6039630B400311D08293111AE
:10025000321C2F292D090339AD00AE09AF098B13CC
:1002600020303707BB002F08BA005621103037075F
:10027000BB002E08BA00562100303707BB002D08FE
:10028000BA0056218B1785018701B70AB6010930DC
:100290003702031C0829822108003E1C08003E107A
:1002A0001030BB003D08BA00562108008B133A08F5
:1002B00083161C159A003B089B0055309D00AA3000
:1002C0009D009C1464009C1862291C1183128B17DA
:1002D000080008000130BD0008000230BD00080021
:1002E0000430BD0008000830BD0008001030BD001B
:1002F00008002030BD0008004030BD0008008030FC
:10030000BD00080001303D020319080002303D0223
:100310000319080004303D020319080008303D02AB
:100320000319080010303D020319080020303D0277
:100330000319080040303D020319080080303D02D7
:10034000031908000130BD003E1408003E140310DC
:10035000BD0DBD1B3D14BD13822108008F0803197C
:1003600008008F0107303D050319A62A02303D051C
:10037000031D51105408EB3C031805125118C329F2
:10038000D40BCE29C829D4035408C83C031CCE2959
:100390000516F530D4005108013AD10002303D0570
:1003A000031DD1105508E63C03188512D118DB292E
:1003B000D50BE629E029D5035508B93C031CE629ED
:1003C0008516F030D5005108023AD10002303D05C3
:1003D000031D51115608DC3C031805105119F3296F
:1003E000D60BFE29F829D6035608B63C031CFE2975
:1003F0000514E630D6005108043AD10002303D051C
:10040000031DD1115708F03C03188510D1190B2A90
:10041000D70B162A102AD7035708D73C031C162AD5
:100420008514FA30D7005108083AD10002303D0552
:10043000031D51125808E03C03188710511A232A53
:10044000D80B2E2A282AD8035808C13C031C2E2A70
:100450008714EA30D8005108103AD10006303D0523
:10046000031DD1125908D43C03180711D11A3B2A95
:10047000D90B462A402AD9035908A73C031C462A0F
:100480000715DE30D9005108203AD10006303D056D
:10049000031D51135A08BF3C03180710511B532A60
:1004A000DA0B5E2A582ADA035A089C3C031C5E2A9F
:1004B0000714C930DA005108403AD10006303D0532
:1004C000031DD1135B08D73C03188712D11B6B2A7D
:1004D000DB0B762A702ADB035B08BE3C031C762A02
:1004E0008716E130DB005108803AD10006303D0527
:1004F000031D52105C08F13C031807125218832A9E
:10050000DC0B8E2A882ADC035C08CF3C031C8E2A75
:100510000716FB30DC005208013AD20006303D05D8
:10052000031DD2105D08E93C03188711D2189B2ADD
:10053000DD0BA62AA02ADD035D08B23C031CA62A17
:100540008715F330DD005208023AD20018303D051D
:100550000319F62ABD1DB22A54083C3C031CB22ADA
:1005600085018701D40B0800D0034630D4000B303E
:100570005002031DBC2A05160A305002031DC12A71
:10058000851609305002031DC62A05140830500292
:10059000031DCB2A851407305002031DD02A87146F
:1005A00006305002031DD52A071505305002031DE1
:1005B000DA2A071404305002031DDF2A871603309D
:1005C0005002031DE42A071602305002031DE92AD7
:1005D000871501305002031DED2A12305002031C12
:1005E0000800850187010C30D000080020303D054F
:1005F0000319402BD40B012B0508103A85008230DB
:10060000D400D50B082B0508203A85007D30D50095
:10061000D60B0F2B0508013A85007330D600D70B97
:10062000162B0508023A85008730D700D80B1D2B02
:100630000708023A87007730D800D90B242B070827
:10064000043A87006B30D900DA0B2B2B0708013AEC
:1006500087005630DA00DB0B322B0708203A870080
:100660006E30DB00DC0B392B0708103A870088302E
:10067000DC00DD0B402B0708083A87008030DD00E6
:1006800040303D050319B72B5408E63C031805120A
:10069000D40B662B0516F030D4002130DE0703188A
:1006A000642BB130D507FA30D607C830D70764308D
:1006B000D8079630D907BE30DA07AA30DB079A3060
:1006C000DC07C430DD07662B8030BD005508823C56
:1006D00003188512D50B6F2B85168C30D500560864
:1006E000653C03180510D60B782B05146F30D60027
:1006F0005708913C03188510D70B812B85149B302C
:10070000D7005808D73C03188710D80B8A2B8714BA
:10071000E130D8005908503C03180711D90B932B2E
:1007200007155A30D9005A08873C03180710DA0B0E
:100730009C2B07149130DA005B08BD3C031887122C
:10074000DB0BA52B8716C730DB005C08703C031859
:100750000712DC0BAE2B07167A30DC005D08A73CD5
:1007600003188711DD0BB72B8715B130DD00803002
:0E0770003D050319BE2B85018701DE0108003F
:084000000B00030002000600A2
:02400E00CC01E3
:10420000FF00FF00FF00FF00FF00FF00FF00FF00B6
:10421000FF00FF00FF00FF00FF00FF00FF00FF00A6
:104220000100FF00FF00FF00FF00FF00FF00FF0094
:10423000FF00FF00FF00FF00FF00FF00FF00FF0086
:104240001000FF00FF00FF00FF00FF00FF00FF0065
:10425000FF00FF00FF00FF00FF00FF00FF00050060
:10426000FF00FF00FF00FF00FF00FF00FF00FF0056
:10427000FF00FF00FF00FF00FF00FF00FF00FF0046
:10428000FF00FF00FF00FF00FF00FF00FF00FF0036
:10429000FF00FF00FF00FF00FF00FF00FF00FF0026
:1042A000FF00FF00FF00FF00FF00FF00FF00FF0016
:1042B000FF00FF00FF00FF00FF00FF00FF00FF0006
:1042C000FF00FF00FF00FF00FF00FF00FF00FF00F6
:1042D000FF00FF00FF00FF00FF00FF00FF00FF00E6
:1042E000FF00FF00FF00FF00FF00FF00FF00FF00D6
:1042F000FF00FF00FF00FF00FF00FF00FF000000C5
:00000001FF
